:1000000013298030A100FE30A7200130A7207530D1
:10001000A7003030BF28A101A117AF00AF08031D12
:100020001328030114280130AF020310A20CA20C04
:10003000A20CC0302205403EAF07FE30A7202F089B
:10004000A728A101A117AF00FE30A7202F08A728DD
:10005000A401AA00AB01A01124080319A0150530C2
:10006000A3002730A900103041200330A900E83058
:100070004120A90164304120A9010A3041202A0809
:100080004828A8002B08A7002A08A600DD2026087B
:10009000A600A3030319A011240803195228230260
:1000A000031859282608031DA011A0195928303E0D
:1000B000A7280800AD0006118611831606118611C7
:1000C0000F30860583122D08A01884283E30A70023
:1000D0008030BF203330AC0098201330A700883028
:1000E000BF2098206430BE2098206430BE2022308B
:1000F000AC009820283083200C30832006308320E9
:10010000A0142D0884282014AC00201C92288611ED
:10011000033C031C972897200730A700D030BF204E
:10012000031408002014FE3C0319A5288615201C82
:10013000201006150F3086052C08F03986040611AC
:10014000AC0E201898283230BE202D080F29A11B94
:100150005A28080083178001840AFF3E031DAB283C
:100160000F29A901A800FF30A807031CA907031C39
:100170000F290330A700DF30BF20B328A701E83ED6
:10018000A600A709FC30031CC828A6070318C52829
:10019000A6070000A70FC5282618CE28A61CD2281F
:1001A0000000D2280800013EAD000A30A800A901D5
:1001B000DD20AD0BD8282A080800AB01AA011030B9
:1001C000AC00270DAA0DAB0D2808AA022908031CB4
:1001D000290FAB020318F3282808AA0729080318D7
:1001E000290FAB070310A60DA70DAC0BE1282608BD
:1001F0000F291030B000A701A601AD0CAC0C031CF8
:1002000007292808A60729080318290FA707A70CFC
:10021000A60CAB0CAA0CB00BFD282A080F298313DF
:10022000831203130800A00107309F00E0308316FB
:100230008500FF30860081138312850186012030FE
:1002400084006030AB20A03084005030AB202030E0
:1002500084003030AA20C830B120012077305A20E5
:100260005A205A202E305A2070305A2069305A2095
:1002700063305A2062305A208030A100C0302120E3
:1002800061305A2073305A2069305A2063305A2026
:100290002E305A206E305A206C305A200B30A90074
:1002A000B830B220012044305A2043305A20463022
:1002B0005A2031305A2036305A204E305A204C3095
:1002C0005A2045305A208030A100C23021205630BB
:1002D0005A202D305A2032305A200730A900D03011
:1002E000B220012044305A2069305A2073305A20FD
:1002F00070305A206C305A2061305A2079305A20A0
:100300008030A100C030212061305A2066305A2050
:1003100072305A2065305A2067305A2065305A2092
:100320006C305A2065305A206E305A2086189E292B
:10033000851F9C2905149D290510962901205330FD
:100340005A2069305A2067305A206E305A20613066
:100350005A205A206C305A208030A100C030212011
:100360007A305A206F305A2065305A206B305A202C
:1003700065305A206E305A204914831605128312B4
:100380000512442AC2013B03A500C8014808250202
:10039000031CDA29FD21C91CD7294808A200A6019F
:1003A000A20A0314A60DA20BD2292608C204C80A69
:1003B000031DC6294208B100B201B20CB10CB20C47
:1003C000B10CB20CB10CB20CB10C0F30B20531084B
:1003D000AC003208AD000A30A800A901F920B10034
:1003E0002B08B2004208B300B4010F30B30500304F
:1003F000B40531083307C2000800B801B901061876
:10040000122A0130B120B80A0319B90A0B30390297
:10041000031C112A031D102AB9303802031C112AAB
:10042000882CFF299B30B120831006188314831871
:10043000C914831CC910491C312A4308B100B201F8
:100440000310B10DB20DB10DB20DB10DB20D3108E9
:10045000A6003208A7003A30A800A901DD20BC00A0
:100460003A2A03014919013EC918013A03194911F1
:10047000031D4915C30A85140130A900F430B220C8
:100480008510F030B1200800BA01C3014912491AA1
:10049000D82AB801B901061C5E2AB80A0319B90A9C
:1004A0000130B120AF303902031C5D2A031D5C2AE4
:1004B000C9303802031C5D2A882C4B2AB801B901C7
:1004C0000618902AB80A0319B90A0A30B120491847
:1004D000842A38080B3A3904031D6F2A832A380806
:1004E000193A3904031D762A8514832A38084B3AB1
:1004F0003904031D7D2A8510832A3808FA3A390405
:10050000031D832A882C8F2A11303902031C8F2A5D
:10051000031D8E2A95303802031C8F2A882C602AEE
:1005200041303A02031C952A882CBA0AB908031DE7
:100530009D2A65303802031C9E2A4916491CD72A79
:100540003A08B100B2010310B10DB20DB10DB20DF8
:10055000B10DB20D3108A6003208A7004130A80045
:10056000A901DD20BC008030A100212053305A2099
:1005700069305A2067305A206E305A2061305A2034
:100580005A206C305A2020305A20C0302120673049
:100590005A2065305A2076305A206F305A206E30FB
:1005A0005A2064305A2065305A206E305A20472A2B
:1005B000491CFE2A012049305A206E305A206930E9
:1005C0005A2074305A2069305A2061305A206C30D9
:1005D0005A2069305A208030A100C0302120733069
:1005E0005A2065305A2072305A2065305A206E30B9
:1005F0005A202E305A205A205A205C2B0330BC003F
:100600000230A2003C080B20A101C91D162B3B3073
:10061000400203180D2BC00A152BC00117304402ED
:100620000318142BC40A152BC4011A2B4108C0004F
:100630004508C400051B2A2BC408031D222B0C30BF
:10064000C600292B0D304402031C292B0C30440218
:10065000C6002E2B4408C60020305A200A3046021D
:100660000318342B20305A208030A100460828205F
:100670003A305A200230A40040082920051B4A2B9A
:100680000C3044020318472B61305A20492B70303C
:100690005A204A2B0130C008031D0030B5001E301F
:1006A00040020130031D0030B504013086180301FB
:1006B000B50403195C2B612C491E5F2CFD21013010
:1006C000C8000F3048020318692BFD21C80A031D1A
:1006D000612B4911C911FD21FD21FD21C91C722B7E
:1006E0000514732B05101230C8001430480203188B
:1006F0007D2BFD21C80A031D752BFD210730BB0092
:10070000C2214208C100FD21491D872BC9150630B1
:10071000BB00C2214208C500FD21491D902BC9150F
:100720000630BB00C2214208BD000330BB00C2211D
:100730004208C7000530BB00C2214208BF00083094
:10074000BB00C2214208BE00FD21491DA82BC915CE
:10075000491CAE2BC919AD2B49100120C9195E2CBB
:100760008030A10021200230A4003D082920203043
:100770005A2001303F02031DC42B6A305A206130D9
:100780005A206E305A203C2C02303F02031DCF2BE2
:1007900066305A2065305A2062305A203C2C033093
:1007A0003F02031DDA2B6D305A2072305A2074300C
:1007B0005A203C2C04303F02031DE52B61305A20A7
:1007C00070305A2072305A203C2C05303F02031DF5
:1007D000F02B6D305A2065305A2069305A203C2C5D
:1007E00006303F02031DFB2B6A305A2075305A2019
:1007F0006E305A203C2C07303F02031D062C6A3015
:100800005A2075305A206C305A203C2C08303F0258
:10081000031D112C61305A2075305A2067305A2040
:100820003C2C09303F02031D1C2C73305A206530CC
:100830005A2070305A203C2C0A303F02031D272CCE
:100840006F305A206B305A2074305A203C2C0B30B9
:100850003F02031D322C6E305A206F305A20763002
:100860005A203C2C0C303F02031D3C2C64305A2093
:1008700065305A2063305A20051B522C20305A20F4
:100880008030A100A4013E08A600A7010130D320BA
:10089000AA00AB012B20C03021200130A4003E086B
:1008A00029205E2C20305A2027305A208030A10089
:1008B000C03021200230A4003E082920602C882C62
:1008C000442A851F682C83160512831205126A2C90
:1008D0008316051683129B30B1200130C008031D1A
:1008E0000030B500013086180301B5040319792CD6
:1008F0000515851585140130A900F430B2200511C5
:10090000851185100130A9004A30B220C30A5F2B3F
:10091000012047305A2065305A205A206E305A2024
:1009200020305A2073305A2069305A2067305A20BC
:100930008030A100C03021206E305A2061305A2012
:100940005A206C305A20203084006030AB20A03018
:1009500084005030AB20203084003030AA20831037
:10096000061883148318C916831CC91203010618BC
:10097000013EC91A013C031DC32CB60A0319B70A6C
:100980000130B120B62C0301C91A0130013A031914
:10099000C912031DC91603010618013EC91A013CFC
:1009A000031DD82CB60A0319B70A0130B120CB2C8D
:1009B00003303702DE30031936020318A32C491422
:0409C000442AE12CB8
:02400E00503F21
:00000001FF
